:020000040000FA
:10000000012830209E200D20D720D7204E20B6007A
:1000100056208320D720D72006288030BE2051309C
:10002000B7205230B7205030B7202030B7205030A2
:10003000B7206F30B7207730B7206530B7207230E7
:10004000B7202030B7207630B7202E30B7203030A0
:10005000B7202E30B7203030B7203130B72008001D
:1000600061308F00830185010730990083160930C4
:100070008500013091000030870010309F0083120E
:1000800001309F000B13FF308700F63085003030C1
:10009000B200B300B4002D30B000080001309F0062
:1000A000E9209F149F1852281E08080002308A0079
:1000B00036080022A40000308A002408692003309A
:1000C0008A0036080023A40000308A002408762025
:1000D0000800A400B7002D3024182B30B008A40C61
:1000E000A40CA40C240C8020B2000800A4008020E2
:1000F000B300A40CA40CA40C240C8020B4000800B1
:100100000F39303E0800C030BE202030B7202030EC
:10011000B7203008B7203408B7203308B7202E3076
:10012000B7203208B7202030B7206430B7204230E3
:10013000B7206D30B7205730B7200800DD20DD2014
:10014000DD200330D020DD200330D020DD2003303F
:10015000D020DD200230D020DD202E30BE2008301F
:10016000BE200C30BE200630BE20C5200800B500E1
:10017000350ECD203508CD20E9200800B500350E1C
:10018000D0203508D020E92008000130BE20DD2035
:1001900008000230BE20DD2008000F391038D128B9
:1001A0000F398700203887001F39870008001E306C
:1001B000A300DD20A30BD92808003230A100E920DC
:1001C000A10BDF2808000A30A100E920A10BE528D7
:1001D00008001830A0000000A00BEB280000000071
:0E01E00008000C30A0000000A00BF32808005F
:10040000B61F042A361BBF3082070234023402347E
:100410000234023402340234023402340034003430
:10042000003400340034003400340034003400342C
:10043000003400340034003400340034003400341C
:10044000003400340034003400340034003400340C
:1004500000340034003400340034003400340034FC
:1004600000340034003400340034003400340034EC
:1004700000340034003400340034003400340034DC
:1004800000340034003400340034003400340034CC
:1004900000340034003400340034003401340134BA
:1004A00001340134013401340134013401340134A4
:1004B000013401340134013403340334033403348C
:1004C0000334033403340334033403340334033474
:1004D0000334033403340334033403340334033464
:1004E0000334033403340334033403340334033454
:1004F0000334033403340334033403340334033444
:100500000334033403340334033403340334033433
:100510000334033403340334033403340334033423
:100520000334033403340334033403340334033413
:100530000334033403340334033403340334033403
:1005400003340334033403340334033403340334F3
:1005500003340334033403340334033403340334E3
:1005600003340334033403340334033403340334D3
:1005700003340334033403340334033403340334C3
:0C05800003340334033403340334033425
:10060000B61F042B361BBF30820755345534553482
:100610005534553455345534553455345534543493
:1006200053345334523452345034473445344334C1
:100630004234413440344034393438343734363439
:100640003534353434343334323431343034303476
:1006500029342834273426342634253425342534C7
:1006600024342334223421342034203419341834EF
:100670001834173416341534153414341334123432
:100680001134103410340934093408340734063472
:1006900005340434033402340234013400340034A9
:1006A0000434063408341034103400340034003478
:1006B000003400340034003400340034003400349A
:1006C000003400340034003400340034003400348A
:1006D000003400340034003400340034003400347A
:1006E000003400340034003400340034003400346A
:1006F000003400340034003400340034003400345A
:100700000034003400340034003400340034003449
:100710000034003400340034003400340034003439
:100720000034003400340034003400340034003429
:100730000034003400340034003400340034003419
:100740000034003400340034003400340034003409
:1007500000340034003400340034003400340034F9
:1007600000340034003400340034003400340034E9
:1007700000340034003400340034003400340034D9
:0C07800000340034003400340034003435
:02400E00C433B9
:00000001FF
